:100000000C9435000C945D000C945D000C945D0024
:100010000C945D000C945D000C945D000C945D00EC
:100020000C945D000C945D000C945D000C945D00DC
:100030000C945D000C945D000C945D000C945D00CC
:100040000C9471010C945D000C94E1010C94BB01C3
:100050000C945D000C945D000C945D000C945D00AC
:100060000C945D000C945D009E0211241FBECFEF26
:10007000D8E0DEBFCDBF11E0A0E0B1E0E0EBF5E0FD
:1000800002C005900D92A231B107D9F721E0A2E19B
:10009000B1E001C01D92A83BB207E1F710E0C5E353
:1000A000D0E004C02197FE010E94CB02C433D107E7
:1000B000C9F70E9413020C94D6020C940000CF9250
:1000C000DF92EF92FF920F931F93CF93DF936C0118
:1000D0007A018B01C0E0D0E0CE15DF0581F0D801B8
:1000E0006D918D01D601ED91FC910190F081E02D93
:1000F000C6010995892B11F02196EECF7E01C7012B
:10010000DF91CF911F910F91FF90EF90DF90CF90F3
:100110000895089580E090E00895FC01538D448D8A
:10012000252F30E0842F90E0821B930B541710F0A2
:10013000CF96089501970895FC01918D828D9817AF
:1001400061F0828DDF01A80FB11D5D968C91928DBB
:100150009F5F9F73928F90E008958FEF9FEF0895B8
:10016000FC01918D828D981731F0828DE80FF11D81
:10017000858D90E008958FEF9FEF0895FC01918D9C
:10018000228D892F90E0805C9F4F821B91098F7395
:100190009927089582E191E00E94BE0021E0892B19
:1001A00009F420E0822F0895FC01848DDF01A80F5F
:1001B000B11DA35ABF4F2C91848D90E001968F738F
:1001C0009927848FA689B7892C93A089B1898C91AE
:1001D000837080648C93938D848D981306C00288FD
:1001E000F389E02D80818F7D80830895EF92FF92C7
:1001F0000F931F93CF93DF93EC0181E0888F9B8D4A
:100200008C8D981305C0E889F989808185FD26C009
:10021000F62E0B8D10E00F5F1F4F0F731127E02E8E
:100220008C8DE8120CC00FB607FCFACFE889F9896B
:10023000808185FFF5CFCE010E94D400F1CF8B8D58
:10024000FE01E80FF11DE35AFF4FF0829FB7F894CB
:100250000B8FEA89FB89808180620AC09FB7F8947E
:10026000EE89FF896083E889F989808183708064E1
:1002700080839FBF81E090E0DF91CF911F910F912C
:10028000FF90EF900895CF93DF93EC01888D882342
:10029000C9F0EA89FB89808185FD05C0A889B989F3
:1002A0008C9186FD0FC00FB607FCF5CF808185FFCE
:1002B000F2CFA889B9898C9185FFEDCFCE010E943C
:1002C000D400E7CFDF91CF91089580E090E0892BB3
:1002D00029F00E94CA0081110C94000008950E9428
:1002E000D1021F920F920FB60F9211242F933F93BA
:1002F0008F939F93AF93BF938091B4019091B50179
:10030000A091B601B091B7013091B30123E0230F62
:100310002D3720F40196A11DB11D05C026E8230F3D
:100320000296A11DB11D2093B3018093B401909357
:10033000B501A093B601B093B7018091AF01909140
:10034000B001A091B101B091B2010196A11DB11D02
:100350008093AF019093B001A093B101B093B2012B
:10036000BF91AF919F918F913F912F910F900FBEB1
:100370000F901F9018951F920F920FB60F92112495
:100380002F933F934F935F936F937F938F939F939D
:10039000AF93BF93EF93FF9382E191E00E94D4006B
:1003A000FF91EF91BF91AF919F918F917F916F914D
:1003B0005F914F913F912F910F900FBE0F901F9023
:1003C00018951F920F920FB60F9211242F938F93AF
:1003D0009F93EF93FF93E0912201F091230180819D
:1003E000E0912801F091290182FD12C09081809155
:1003F0002B018F5F8F7320912C01821751F0E091B8
:100400002B01F0E0EE5EFE4F958F80932B0101C033
:100410008081FF91EF919F918F912F910F900FBE4F
:100420000F901F901895789484B5826084BD84B530
:10043000816084BD85B5826085BD85B5816085BDDF
:1004400080916E00816080936E0010928100809197
:10045000810082608093810080918100816080931F
:100460008100809180008160809380008091B10044
:1004700084608093B1008091B00081608093B0006F
:1004800080917A00846080937A0080917A00826003
:1004900080937A0080917A00816080937A008091C5
:1004A0007A00806880937A001092C100E091220166
:1004B000F091230182E08083E0911E01F0911F0101
:1004C0001082E0912001F091210180E1808310925F
:1004D0002A01E0912601F091270186E08083E091D6
:1004E0002401F0912501808180618083E0912401C5
:1004F000F0912501808188608083E0912401F09152
:100500002501808180688083E0912401F09125019C
:1005100080818F7D808382E191E00E94BE00181669
:1005200019064CF482E191E00E949C00682F82E160
:1005300091E00E94F6000E946501EDCFE2E1F1E05A
:100540001382128288EE93E0A0E0B0E0848395836A
:10055000A683B78384E091E09183808385EC90E06B
:100560009587848784EC90E09787868780EC90E07D
:10057000918B808B81EC90E0938B828B82EC90E06E
:10058000958B848B86EC90E0978B868B118E128EE8
:10059000138E148E0895EE0FFF1F0590F491E02D39
:1005A000099481E090E0F8940C94D602F894FFCF7F
:1005B00000000000F6005F008D004301BE009C00BB
:0205C000B00089
:00000001FF
